:020000040000FA
:10000000CEEF1AF012001200E9EF00F0120001002A
:10001000EE35000000010000A2000000400EE66E78
:10002000E66A740EE66EE9EC19F0E552E552E55227
:100030009F8AD08E9D9AF29CF29E1200D9CFE6FF45
:10004000E1CFD9FF020EE126DE6ADD6AFD0EDBCFCD
:10005000F6FFFE0EDBCFF7FF0800F55015E0FD0EB2
:10006000DBCFF6FFFE0EDBCFF7FF0800F550E66EA4
:1000700055D8E552DF2A010E01E3DB2AFD0EDB2A0B
:10008000FE0E01E3DB2AE2D7DECF00F0DDCF01F088
:1000900000C0F3FF01C0F4FF020EE15C03E200D0F8
:1000A000E16AE552E16EE552E7CFD9FF1200D9CF00
:1000B000E6FFE1CFD9FF020EE126DE6ADD6AFD0E22
:1000C000DBCFE9FFFE0EDBCFEAFFEF5014E0FD0EC1
:1000D000DBCFE9FFFE0EDBCFEAFFEF50E66E1ED866
:1000E000E552DF2A010E01E3DB2AFD0EDB2AFE0EBC
:1000F00001E3DB2AE4D7DECF00F0DDCF01F000C062
:10010000F3FF01C0F4FF020EE15C03E200D0E16AFC
:10011000E552E16EE552E7CFD9FF1200D9CFE6FFF5
:10012000E1CFD9FFACA2FED7FE0EDBCFE6FF95EC08
:100130001AF0E552E552E7CFD9FF12000D0EE66E38
:10014000EDDFE5520A0EE66EE9DFE5521200D9CF87
:10015000E6FFE1CFD9FFE65207010451021902E19F
:100160000551031901E1F8D702C7E9FF03C7EAFF08
:10017000022B000E0323EFCFDFFF980E025D010E6E
:10018000035904E3700E026F010E036FDF5000D0BD
:10019000E552E552E7CFD9FF120007017A51EA6A2A
:1001A000000FE96E060EEA22EF50836E740EE96EC0
:1001B000070EEA6E7851EE24786F7951EE20796F50
:1001C0007A51EE207A6F7B51EE207B6F1151E5E082
:1001D0001200DACFE4FFE2CFDAFFE9CFE4FFEACFA3
:1001E000E4FFF6CFE4FFF7CFE4FFF5CFE4FFF3CF72
:1001F000E4FFF4CFE4FFFACFE4FF00EE18F0140EB2
:10020000E80403E3EECFE4FFFBD700EE00F0180EA6
:10021000E80403E3EECFE4FFFBD7E6529EAA34D016
:100220005AEC1AF00701116FABA407D0AB9E7D8189
:100230000F2B000E1023AB8E01D07D91ABA207D007
:10024000AB987D83AB880D2B000E0E2301D07D93E0
:10025000ACA2FED781B205D011C7E6FF95EC1AF02B
:10026000E552070104C7E9FF05C7EAFF042B000EAA
:10027000052311C7EFFF980E045D010E055904E335
:10028000700E046F010E056FE55200EE17F0180EA8
:10029000E80403E3E5CFEDFFFBD700EE2BF0140EEF
:1002A000E80403E3E5CFEDFFFBD7E5CFFAFFE5CFA9
:1002B000F4FFE5CFF3FFE5CFF5FFE5CFF7FFE5CF9F
:1002C000F6FFE5CFEAFFE5CFE9FFE5CFDAFF110062
:1002D000D9CFE6FFE1CFD9FFFF0EE76EFD0EDBCFF2
:1002E00000F0FE0EDBCF01F0E7500016016A00506F
:1002F000A96EFD0EDBCF00F0FE0EDBCF01F001C0DA
:1003000000F0016A030E0014AA6EA69EA69CA680A9
:10031000E80EE66E030EE66EE66AE66A52EC07F059
:10032000E552E552E552E552A85000D0E552E7CF3C
:10033000D9FF1200D9CFE6FFE1CFD9FF020EE126A7
:10034000FD0EDBCF00F0FE0EDBCF01F001C000F0B0
:10035000016A030E0014AA6EFF0EE76EFD0EDBCFDE
:1003600000F0FE0EDBCF01F0E7500016016A0050EE
:10037000A96EFC0EDB50A86EA69EA684A69CF2AECB
:1003800004D0F29E010EDE6EDD6A550EA76EAA0E37
:10039000A76EA682A1A8FED7A198A694D9CFE9FFFF
:1003A000DACFEAFF010EEE1801E1ED5001E1F28E25
:1003B000020EE15C02E2E16AE552E16EE552E7CF4E
:1003C000D9FF1200D9CFE6FFE1CFD9FFFB0EDBCF7B
:1003D000E9FFFC0EDBCFEAFFEF5022E0FB0EDBCFA4
:1003E000E9FFDB2AFC0EDBCFEAFF01E3DB2AEF505B
:1003F000E66ED950FD0FE96EFF0EDA20EA6EEECF01
:1004000000F0EDCF01F0020EEE26000EEF2200C04C
:10041000E6FF01C0E6FF8EDFE552E552E552D6D792
:10042000E552E7CFD9FF1200D9CFE6FFE1CFD9FFE0
:10043000020EE126D950FD0FE96EFF0EDA20EA6EBA
:10044000FF0ED880EE54030EED5401E223D0FD0ED2
:10045000DBCFE6FFFE0EDBCFE6FF3ADFE552E552EB
:10046000DE6EDD6AD9CFE9FFDACFEAFFEE50ED109C
:1004700001E110D0DFCFE6FF51DEE552FD0EDB2AB1
:10048000FE0E01E3DB2AD9CFE9FFDACFEAFFEE5017
:10049000ED10D0E1E80EE66E030EE66EE66AE66A5F
:1004A00052EC07F0E552E552E552E552020EE15CEE
:1004B00002E2E16AE552E16EE552E7CFD9FF1200B0
:1004C000D9CFE6FFE1CFD9FF040EE1260701600E88
:1004D000006F010E016F00C7E6FF01C7E6FFFD0ECA
:1004E000DBCFE6FFFE0EDBCFE6FF0DEC15F0E552AD
:1004F000E552E552E55200C7E6FF01C7E6FFDBEC37
:1005000019F0E552E552F3CFDEFFF4CFDDFFD9CF8E
:10051000E9FFDACFEAFF020EEECFDBFF030EEDCFED
:10052000DBFF020EDBCF00F0030EDBCF01F0040E89
:10053000005C000E01580AE2300EE66EEFDDE55277
:10054000020EDB2A030E01E3DB2AEBD700C7E6FF2E
:1005500001C7E6FFACDDE552E552F3CFDEFFF4CF95
:10056000DDFF040EE15C02E2E16AE552E16EE55274
:10057000E7CFD9FF1200D9CFE6FFE1CFD9FF0E0EAA
:10058000E126F90EDBCFDEFFDBCFDDFFF80EDB501F
:10059000000802E3070E08D0F80EDB50160802E24E
:1005A000170E02D0F80EDB28E66ED950080FE96E60
:1005B000DACFEAFFE552E750EE6EED6A020EDB6A33
:1005C000030EDB6AFB0EDBCF00F0FC0EDBCF01F08D
:1005D000FD0EDBCF02F0FE0EDBCF03F0226A236AB2
:1005E000246A256A00C01DF001C01EF002C01FF081
:1005F00003C020F0D7EC10F0010A33E1F90EDBCF95
:10060000E9FFDB2AFA0EDBCFEAFF01E3DB2A2D0E3E
:10061000EF6EFB0EDBCF00F0FC0EDBCF01F0FD0E2A
:10062000DBCF02F0FE0EDBCF03F0226A236A800EDE
:10063000246EBF0E256E00C01DF001C01EF002C06A
:100640001FF003C020F0FBEC0FF0FB0E1DC0DBFF22
:10065000FC0E1EC0DBFFFD0E1FC0DBFFFE0E20C028
:10066000DBFFFB0EDBCF00F0FC0EDBCF01F0FD0E5D
:10067000DBCF02F0FE0EDBCF03F0226A236A246A8E
:10068000256A00C01DF001C01EF002C01FF003C0AB
:1006900020F0CEEC10F0010A4AE1FB0EDBCF00F0B7
:1006A000FC0EDBCF01F0FD0EDBCF02F0FE0EDBCF48
:1006B00003F0226A236A800E246E3F0E256E00C06E
:1006C0001DF001C01EF002C01FF003C020F0D7ECE7
:1006D00010F0010A2CE1006A016A200E026E410E40
:1006E000036ED950FB0FE96EFF0EDA20EA6EEECFF3
:1006F0001DF0EECF1EF0EECF1FF0EFCF20F000C0C8
:1007000022F001C023F002C024F003C025F0FBEC6E
:100710000FF020C0EDFF1FC0EDFF1EC0EDFF1DC09C
:10072000EFFF020EDB06030E01E2DB06B6D7FB0E7F
:10073000DBCF00F0FC0EDBCF01F0FD0EDBCF02F0D3
:10074000FE0EDBCF03F0226A236A200E246E410ED8
:10075000256E00C01DF001C01EF002C01FF003C0D6
:1007600020F0D7EC10F0010A2EE0FB0EDBCF00F0FA
:10077000FC0EDBCF01F0FD0EDBCF02F0FE0EDBCF77
:1007800003F0226A236A200E246E410E256E00C0FB
:100790001DF001C01EF002C01FF003C020F0A8EC45
:1007A0000FF0FB0E1DC0DBFFFC0E1EC0DBFFFD0EBD
:1007B0001FC0DBFFFE0E20C0DBFF020EDB2A030E94
:1007C00001E3DB2AB4D7020EDBCF00F0030EDBCF50
:1007D00001F0D950080FE96EDACFEAFF0050EE269B
:1007E0000150ED22010EF36E040EF3CFDBFF050E78
:1007F000DB6A040EDBCF1EF0050EDBCF1FF0E3EC4F
:100800000EF00A0E1DC0DBFF0B0E1EC0DBFF0C0E30
:100810001FC0DBFF0D0E20C0DBFF040EDBCF00F09E
:10082000050EDBCF01F0080EDBCF02F0090EDBCFA7
:1008300003F001500318E8AE02D0033404D0025094
:10084000005C035001582EE20A0EDBCF00F00B0EC5
:10085000DBCF01F00C0EDBCF02F00D0EDBCF03F08F
:10086000226A236A200E246E410E256E00C01DF000
:1008700001C01EF002C01FF003C020F0A8EC0FF072
:100880000A0E1DC0DBFF0B0E1EC0DBFF0C0E1FC0CF
:10089000DBFF0D0E20C0DBFF040EDB2A050E01E39B
:1008A000DB2ABBD70A0EDBCF04F00B0EDBCF05F043
:1008B0000C0EDBCF06F00D0EDBCF07F0226A236AA9
:1008C000246A400E256E04C01DF005C01EF006C04F
:1008D0001FF007C020F0A8EC0FF01DC000F01EC0F4
:1008E00001F01FC002F020C003F0D950FB0FE96EE9
:1008F000FF0EDA20EA6EEECF1DF0EECF1EF0EECF47
:100900001FF0EFCF20F000C022F001C023F002C0A2
:1009100024F003C025F012EC0FF020C0EDFF1FC043
:10092000EDFF1EC0EDFF1DC0EFFFFB0EDBCF00F0A3
:10093000FC0EDBCF01F0FD0EDBCF02F0FE0EDBCFB5
:1009400003F0226A236A200E246E410E256E00C039
:100950001DF001C01EF002C01FF003C020F0D7EC54
:1009600010F0010A13E0FB0EDB6AFC0EDB6A800E5E
:10097000F36EFD0EF3CFDBFF3F0EF36EFE0EF3CFF3
:10098000DBFF020EDB2A030E01E3DB2A020EDBCFC4
:1009900000F0030EDBCF01F00001800E01145FE0D8
:1009A000F90EDBCFE9FFDB2AFA0EDBCFEAFF01E32A
:1009B000DB2A300EEF6EF90EDBCFE9FFDB2AFA0EF1
:1009C000DBCFEAFF01E3DB2A2E0EEF6E080EDBCF52
:1009D00000F0090EDBCF01F0800E011414E0020ECE
:1009E000DBCF02F0030EDBCF03F0080EDB50025C1E
:1009F000006E090EDB500358016E020E00C0DBFFD3
:100A0000030E01C0DBFF040EDB68050EDB68040E7D
:100A1000DBCF00F0050EDBCF01F0020EDBCF02F0E2
:100A2000030EDBCF03F003500118E8AE02D001340F
:100A300004D00050025C0150035811E2F90EDBCFE4
:100A4000E9FFDB2AFA0EDBCFEAFF01E3DB2A300EF7
:100A5000EF6E040EDB06050E01E2DB06D8D7040EAE
:100A6000DB6A050EDB6A040EDBCF00F0050EDBCF80
:100A700001F0080EDBCF02F0090EDBCF03F00150CE
:100A80000318E8AE02D0033404D00250005C0350D7
:100A9000015801E3ACD0FB0EDBCF1DF0FC0EDBCF29
:100AA0001EF0FD0EDBCF1FF0FE0EDBCF20F068EC5A
:100AB00010F0060E1EC0DBFF070E1FC0DBFF300E5E
:100AC000E76E060EDBCF00F0070EDBCF01F0E7503C
:100AD0000026000E0122F90EDBCFE9FFDB2AFA0E19
:100AE000DBCFEAFF01E3DB2A00C0EFFF040EDBCF20
:100AF00000F0050EDBCF01F0020EDB50001803E121
:100B0000030EDB5001180BE1F90EDBCFE9FFDB2A06
:100B1000FA0EDBCFEAFF01E3DB2A2E0EEF6E060EA4
:100B2000DBCF1EF0070EDBCF1FF0E3EC0EF00A0E5A
:100B30001DC0DBFF0B0E1EC0DBFF0C0E1FC0DBFF5A
:100B40000D0E20C0DBFF1DC000F01EC001F01FC055
:100B500002F020C003F0D950FB0FE96EFF0EDA203F
:100B6000EA6EEECF1DF0EECF1EF0EECF1FF0EFCF0E
:100B700020F000C022F001C023F002C024F003C026
:100B800025F011EC0FF020C0EDFF1FC0EDFF1EC0DF
:100B9000EDFF1DC0EFFF006A016A200E026E410EDC
:100BA000036ED950FB0FE96EFF0EDA20EA6EEECF2E
:100BB0001DF0EECF1EF0EECF1FF0EFCF20F000C003
:100BC00022F001C023F002C024F003C025F0FBECAA
:100BD0000FF020C0EDFF1FC0EDFF1EC0EDFF1DC0D8
:100BE000EFFF040EDB2A050E01E3DB2A3CD7F90EEA
:100BF000DBCFE9FFFA0EDBCFEAFFEF6A0E0EE15C16
:100C000002E2E16AE552E16EE552E7CFD9FF120058
:100C1000D9CFE6FFE1CFD9FF060EE12607017C9D83
:100C2000FB0EDBCF1DF0FC0EDBCF1EF0FD0EDBCF8D
:100C30001FF0FE0EDBCF20F097EC10F01CC0DEFFA3
:100C40001DC0DEFF1EC0DEFF1FC0DDFFDD52DD5216
:100C5000FB0EDBCF04F0FC0EDBCF05F0FD0EDBCF8F
:100C600006F0FE0EDBCF07F0F90EDBCF1EF0FA0E1A
:100C7000DBCF1FF0E3EC0EF01DC008F01EC009F042
:100C80001FC00AF020C00BF008C022F009C023F0FA
:100C90000AC024F00BC025F004C01DF005C01EF0F2
:100CA00006C01FF007C020F0FBEC0FF01DC000F0E5
:100CB0001EC001F01FC002F020C003F0F90EDBCF10
:100CC00014F0FA0EDBCF15F0166A176A15AE02D0D3
:100CD0001668176814C01CF015C01DF016C01EF071
:100CE00017C01FF0DFCF21F0010EDBCF22F0020E84
:100CF000DBCF23F0030EDBCF24F022EC1AF018C078
:100D000010F019C011F01AC012F01BC013F010C07F
:100D10001CF011C01DF012C01EF013C01FF0F8EC43
:100D20000EF01DC00CF01EC00DF01FC00EF020C054
:100D30000FF00CC022F00DC023F00EC024F00FC045
:100D400025F000C01DF001C01EF002C01FF003C05E
:100D500020F011EC0FF068EC10F0040E1EC0DBFF69
:100D6000050E1FC0DBFF1E0EE66E010EE66ED9CF2C
:100D7000E9FFDACFEAFFEECFE6FFEECFE6FFEECFF8
:100D8000E6FFEFCFE6FFA7EC15F0006E060EE15E82
:100D900000501E0EE66E010EE66E57EC00F0E552B6
:100DA000E552F3CF16F7F4CF17F72E0EE66E8EEC62
:100DB00000F0E552040EDBCFE6FF050EDBCFE6FFC9
:100DC00060EC02F0E552E552060EE15C02E2E16AF7
:100DD000E552E16EE552E7CFD9FF1200D9CFE6FF29
:100DE000E1CFD9FFE652800EDF6EDF50000813E23C
:100DF000FE0EDB50DF1406E0310EE66E8EEC00F0E6
:100E0000E55205D0300EE66E8EEC00F0E552DF4084
:100E10007F0BDF6EEAD7E552E552E7CFD9FF12002C
:100E2000D9CFE6FFE1CFD9FF020EE126FE0EDB505F
:100E3000F00BE8380F0B300FDF6EDF50390803E29C
:100E4000070EDF24DF6EFE0EDB500F0B300FE76E58
:100E5000010EE7CFDBFFDB5039080AE2070E006E18
:100E6000010EDBCFE7FF0050E726010EE7CFDBFFE7
:100E7000DFCFE6FF8EEC00F0E552010EDBCFE6FFA0
:100E80008EEC00F0E552680EE66E8EEC00F0E55256
:100E9000020EE15C02E2E16AE552E16EE552E7CF63
:100EA000D9FF1200D9CFE6FFE1CFD9FFFB0EDBCF90
:100EB0001DF0FC0EDBCF1EF0FD0EDBCF1FF0FE0E93
:100EC000DBCF20F02034000E201809E6D880000E79
:100ED0001D54000E1E54000E1F54000E20540CE230
:100EE000D950FB0FE96EFF0EDA20EA6EEE06000E17
:100EF000EE5AEE5AEE5ADAD7E552E7CFD9FF120092
:100F0000D9CFE6FFE1CFD9FF020EE126DE6ADD6A26
:100F1000DECF00F0DDCF01F0FE0EDB50000101AEB0
:100F200002D0D89003D0005C000E01580AE2200ED7
:100F3000E66E8EEC00F0E552DF2A010E01E3DB2ABB
:100F4000E7D7020EE15C02E2E16AE552E16EE552AA
:100F5000E7CFD9FF1200816893680F01396B070E44
:100F6000806E386B3881388338850F0E926E806AB8
:100F700082683A6B800E946E948E949C3B6B956A5B
:100F80003C6B9668606A1200C280C19EC08EC08AA7
:100F9000C088C096C094C082C090C196C194C192CE
:100FA000C1901200D9CFE6FFE1CFD9FF040EE126B0
:100FB000FD0EDBCF00F0FE0EDBCF01F0D890003647
:100FC0000136D89000360136010E0024C26E0A0E9A
:100FD000E66EDCEC1AF0E552F5EC1AF0F0EC1AF0E3
:100FE000000901E0FBD7E7EC1AF0F3CFDEFFF4CF06
:100FF000DDFF5EC1E6FF5FC1E6FFDECFE6FFDDCFCE
:10100000E6FF0DEC15F0E552E552E552E5524D0EC6
:10101000E66E8EEC00F0E552FD0EDBCF00F0FE0E2A
:10102000DBCF01F0300E0024E66E8EEC00F0E552CE
:101030003D0EE66E8EEC00F0E5525EC1E6FF5FC14C
:10104000E6FF57EC00F0E552E552020EF3CFDBFF6E
:10105000030EF4CFDBFF880EE66E130EE66EE66A33
:10106000E66A20DFE552E552E552E552DECF00F0B8
:10107000DDCF01F000C0F3FF01C0F4FF040EE15C1E
:1010800003E200D0E16AE552E16EE552E7CFD9FF15
:101090001200CD9ECD9CCD8ACD88CD96CD94CD82AB
:1010A000CD90CC9ECC9ACC92CC909F80D08EDB0EF3
:1010B000E66E0B0EE66E79EC1AF0E552E5529E9064
:1010C000F29CCD909D90F29EF29C1200D9CFE6FF4B
:1010D000E1CFD9FF020EE126DE6ADD6AFB0EDBCF2F
:1010E000F6FFDB2AFC0EDBCFF7FF01E3DB2A08006B
:1010F000F550E66EFD0EDBCFE9FFDB2AFE0EDBCFFF
:10110000EAFF01E3DB2AE552E750EF6EDF2A010E2A
:1011100001E3DB2ADECF00F0DDCF01F0D8900150F3
:1011200004E6000E005C010E0158D8E3020EE15CFB
:1011300002E2E16AE552E16EE552E7CFD9FF120023
:10114000D9CFE6FFE1CFD9FF020EE126DE6ADD6AE4
:10115000FB0EDBCFF6FFDB2AFC0EDBCFF7FF01E354
:10116000DB2A0800F550E66EFF0EE76EFD0EDBCFC2
:1011700000F0FE0EDBCF01F0E7500026000E01224A
:10118000DE50005CE96EDD500158EA6EE552E75032
:10119000EF6EDF2A010E01E3DB2ADECF00F0DDCFA8
:1011A00001F0D890015004E6000E005C010E0158D9
:1011B000CFE3020EE15C02E2E16AE552E16EE55244
:1011C000E7CFD9FF1200980EE66E3A0EE66EE66A99
:1011D000E66A68DEE552E552E552E552BCDE0701FB
:1011E000700E046F010E056F04C702F705C703F701
:1011F00001011E0E5E6F010E5F6F0701786B796B48
:101200007A6B7B6B7D6B7D8D7D897D957D977D91E7
:101210007D930F6B106B0D6B0E6B846B856B0EECFF
:1012200000F00C0EE66E8EEC00F0E552A00EE66EBD
:10123000860EE66E010EE66EE66A34DEE552E55293
:10124000E552E5529EEC00F05EC1E6FF5FC1E6FFAD
:1012500057EC00F0E552E552F3CF16F7F4CF17F74D
:101260009EEC00F002C100F003C101F0026A00C070
:10127000E6FF01C0E6FF02C0E6FF1E0EE66E010EAD
:10128000E66EC2EC19F0036E050EE15E03501E0E11
:10129000E66E010EE66E57EC00F0E552E552F3CF34
:1012A00016F7F4CF17F79EEC00F0100EE66E270E3F
:1012B000E66EE66AE66AF6DDE552E552E552E5528B
:1012C0001AC100F01BC101F0026A00C0E6FF01C0B4
:1012D000E6FF02C0E6FF1E0EE66E010EE66EC2ECF1
:1012E00019F0036E050EE15E03501E0EE66E010E50
:1012F000E66E57EC00F0E552E552F3CF16F7F4CF67
:1013000017F79EEC00F016C100F017C101F0026A59
:1013100000C0E6FF01C0E6FF02C0E6FF1E0EE66E5B
:10132000010EE66EC2EC19F0036E050EE15E03508D
:101330001E0EE66E010EE66E57EC00F0E552E55229
:10134000F3CF16F7F4CF17F718C100F019C101F069
:10135000026A00C0E6FF01C0E6FF02C0E6FF1E0E03
:10136000E66E010EE66EC2EC19F0036E050EE15E4C
:1013700003501E0EE66E010EE66E57EC00F0E552CD
:10138000E552F3CF16F7F4CF17F7000EE66EE66AD4
:1013900014EC02F0E552E552200EE66EE66A14EC1B
:1013A00002F0E552E552400EE66EE66A14EC02F0F9
:1013B000E552E552600EE66EE66A14EC02F0E55284
:1013C000E552800EE66EE66A14EC02F0E552E55254
:1013D000A00EE66EE66A14EC02F0E552E552C00E8D
:1013E000E66EE66A14EC02F0E552E552E00EE66EB7
:1013F000E66A14EC02F0E552E552E66A010EE66E8A
:1014000014EC02F0E552E552200EE66E010EE66E97
:1014100014EC02F0E552E5529EEC00F014C100F02D
:1014200015C101F0026A00C0E6FF01C0E6FF02C07C
:10143000E6FF1E0EE66E010EE66EC2EC19F0036EBC
:10144000050EE15E03501E0EE66E010EE66E57ECD1
:1014500000F0E552E552F3CF16F7F4CF17F7760E0A
:10146000F66E270EF76E0900F5CF64F70900F5CF89
:1014700065F70900F5CF66F70800F5CF67F7060EA8
:10148000E66E5EC1E6FF5FC1E6FF64C7E6FF65C7C3
:10149000E6FF66C7E6FF67C7E6FFBBEC02F0006E3B
:1014A000070EE15E00505EC1E6FF5FC1E6FF57EC4C
:1014B00000F0E552E552F3CF16F7F4CF17F79EECA4
:1014C00000F062DD0701826B836BE66A010EE66E57
:1014D000760E006E230E016E026A00C0E6FF01C0A8
:1014E000E6FF02C0E6FF000EE66E060EE66E9FEC1B
:1014F00019F0036E070EE15E035012C100F013C134
:1015000001F0026A00C0E6FF01C0E6FF02C0E6FF8C
:101510001E0EE66E010EE66EC2EC19F0036E050EAD
:10152000E15E03501E0EE66E010EE66E57EC00F013
:10153000E552E552F3CF16F7F4CF17F70701786BB2
:10154000796B7A6B7B6B0101E80E9A6F030E9B6FD0
:101550009C6B9D6B9AC11CF09BC11DF09CC11EF041
:101560009DC11FF0F6EC0EF01DC060F71EC061F7C4
:101570001FC062F720C063F7760EF66E270EF76E77
:101580000900F5CF64F70900F5CF65F70900F5CF3D
:1015900066F70800F5CF67F764C722F065C723F048
:1015A00066C724F067C725F060C71DF061C71EF04D
:1015B00062C71FF063C720F0A8EC0FF01DC05CF7F6
:1015C0001EC05DF71FC05EF720C05FF75CC7E6FF77
:1015D0005DC7E6FF5EC7E6FF5FC7E6FFC8EC18F031
:1015E000E552E552E552E5521CC000F01DC001F085
:1015F0001EC002F01FC003F000C01DF001C01EF0AD
:1016000002C01FF003C020F097EC10F01CC074F76C
:101610001DC075F71EC076F71FC077F71E0EE66E69
:10162000010EE66E74C7E6FF75C7E6FF76C7E6FFF4
:1016300077C7E6FFA7EC15F0006E060EE15E0050DE
:101640001E0EE66E010EE66E57EC00F0E552E55216
:10165000F3CF16F7F4CF17F79EEC00F0100EE66EFE
:10166000270EE66EE66AE66A1DDCE552E552E552B3
:10167000E552D08ED09CAB889D8AF28CF28EF28C93
:101680000701806B816B116B07010451021902E1A4
:101690000551031901E100D2A7EC00F00701076F23
:1016A000802B000E812307514D0A01E1C1D1150A9B
:1016B00001E1ABD00A0A01E191D0160A6DE0100AEF
:1016C00049E0170A25E0100A01E0E6D1200EE66E97
:1016D000E66A14EC02F0E552E552E66A010EE66EA7
:1016E000760E006E230E016E026A00C0E6FF01C096
:1016F000E6FF02C0E6FF000EE66E060EE66E9FEC09
:1017000019F0036E070EE15E03500701116BC4D19F
:10171000400EE66EE66A14EC02F0E552E552E66A27
:10172000010EE66E760E006E250E016E026A00C096
:10173000E6FF01C0E6FF02C0E6FF000EE66E060E01
:10174000E66E9FEC19F0036E070EE15E0350070191
:10175000116BA2D1600EE66EE66A14EC02F0E5525F
:10176000E552E66A010EE66E760E006E260E016EFA
:10177000026A00C0E6FF01C0E6FF02C0E6FF000EFD
:10178000E66E060EE66E9FEC19F0036E070EE15E44
:1017900003500701116B80D1800EE66EE66A14ECEF
:1017A00002F0E552E552E66A010EE66E760E006E34
:1017B000240E016E026A00C0E6FF01C0E6FF02C00F
:1017C000E6FF000EE66E060EE66E9FEC19F0036E65
:1017D000070EE15E03500701116B5ED1A00EE66EAD
:1017E000E66A14EC02F0E552E552760EE66E240E3F
:1017F000E66E000EE66E060EE66EA2DCE552E552DF
:10180000E552E5520701116B47D1C00EE66EE66A5C
:1018100014EC02F0E552E552010EC26E0A0EE66EBD
:10182000DCEC1AF0E552F5EC1AF0F0EC1AF00009D5
:1018300001E0FBD7E7EC1AF0F3CF18F7F4CF19F774
:1018400018C71EF019C71FF0E1EC0EF01DC004F020
:101850001EC005F01FC006F020C007F0226A236AF0
:10186000C80E246E420E256E04C01DF005C01EF089
:1018700006C01FF007C020F0FBEC0FF01DC000F009
:101880001EC001F01FC002F020C003F0226A236ACC
:10189000800E246E440E256E00C01DF001C01EF0A7
:1018A00002C01FF003C020F0A8EC0FF01DC068F7C5
:1018B0001EC069F71FC06AF720C06BF70701D890F8
:1018C00019331833D89019331833000ED8801855AF
:1018D000000E195501E3ABD0FF0E185D000E19592B
:1018E00001E3A5D0126B136B1851125D19511359F6
:1018F0000BE2000E1225E96E060E1321EA6EEF6868
:10190000122B000E1323F0D718C712F719C713F7BD
:10191000000E125D010E13590BE2000E1225E96E46
:10192000060E1321EA6EEF6A122B000E1323F0D776
:1019300008C100F009C101F0026A00C0E6FF01C061
:10194000E6FF02C0E6FF1E0EE66E010EE66EC2EC7A
:1019500019F0036E050EE15E03501E0EE66E010ED9
:10196000E66E57EC00F0E552E552F3CF16F7F4CFF0
:1019700017F75EC1E6FF5FC1E6FF18C7E6FF19C7AC
:10198000E6FF0DEC15F0E552E552E552E552090E81
:10199000E66E8EEC00F0E5524D0EE66E8EEC00F039
:1019A000E552300E07011425E66E8EEC00F0E5528C
:1019B0003D0EE66E8EEC00F0E5525EC1E6FF5FC1C3
:1019C000E6FF57EC00F0E552E552F3CF16F7F4CFFF
:1019D00017F7090EE66E8EEC00F0E552020EE66E89
:1019E0005EC1E6FF5FC1E6FF68C7E6FF69C7E6FFC5
:1019F0006AC7E6FF6BC7E6FFBBEC02F0006E070E9E
:101A0000E15E00505EC1E6FF5FC1E6FF57EC00F00B
:101A1000E552E552F3CF16F7F4CF17F7250EE66E31
:101A20008EEC00F0E5529EEC00F00701116B34D013
:101A3000E66A010EE66E14EC02F0E552E55207018B
:101A4000126B136B000E125D010E13590CE2000EA7
:101A50001225E96E060E1321EA6E300EEF6E122B80
:101A6000000E1323EFD7126B136B000E1225E96ED5
:101A7000060E1321EA6E600EEF6E020E126F136BEC
:101A8000000E1225E96E060E1321EA6EEF6A116B45
:101A900003D00701806B816B050ED8808055000E46
:101AA000815501E32DD10D0E075D01E029D1826B37
:101AB000836B126B136B050E125D000E135918E247
:101AC000700E1225E96E010E1321EA6EEF50E66EDC
:101AD000E66AACEC1AF0E552E55207018251F324B4
:101AE000826F8351F420836F122B000E1323E3D7F0
:101AF000050E821901E183512FE09EEC00F010C128
:101B000000F011C101F0026A00C0E6FF01C0E6FF6B
:101B100002C0E6FF1E0EE66E010EE66EC2EC19F084
:101B2000036E050EE15E03501E0EE66E010EE66EBC
:101B300057EC00F0E552E552F3CF16F7F4CF17F764
:101B4000FA0EE66EE66AE66AE66A52EC07F0E552DD
:101B5000E552E552E552C8D0746B756B766B776BC6
:101B60000101756B700EE66E010EE66E62EC14F00C
:101B7000E552E5521CC09AF11DC09BF11EC09CF1BC
:101B80001FC09DF19AC11CF09BC11DF09CC11EF0AD
:101B90009DC11FF0F6EC0EF01DC060F71EC061F78E
:101BA0001FC062F720C063F7760EF66E270EF76E41
:101BB0000900F5CF64F70900F5CF65F70900F5CF07
:101BC00066F70800F5CF67F764C722F065C723F012
:101BD00066C724F067C725F060C71DF061C71EF017
:101BE00062C71FF063C720F0A8EC0FF01DC05CF7C0
:101BF0001EC05DF71FC05EF720C05FF75CC71DF019
:101C00005DC71EF05EC71FF05FC720F097EC10F0B5
:101C10001CC074F71DC075F71EC076F71FC077F79C
:101C20001E0EE66E010EE66E74C7E6FF75C7E6FF90
:101C300076C7E6FF77C7E6FFA7EC15F0006E060E45
:101C4000E15E00501E0EE66E010EE66E57EC00F0EF
:101C5000E552E552F3CF16F7F4CF17F7090EE66E0B
:101C60008EEC00F0E552460EE66E8EEC00F0E5528A
:101C70003D0EE66E8EEC00F0E552010EE66E5EC1A2
:101C8000E6FF5FC1E6FF60C7E6FF61C7E6FF62C728
:101C9000E6FF63C7E6FFBBEC02F0006E070EE15EF5
:101CA00000505EC1E6FF5FC1E6FF57EC00F0E55271
:101CB000E552F3CF16F7F4CF17F7480EE66E8EEC29
:101CC00000F0E5527A0EE66E8EEC00F0E5529EECE6
:101CD00000F074C789F775C788F776C787F70701DB
:101CE000786B796B7A6B7B6B0701700E046F010E5A
:101CF000056F04C702F705C703F7806B816B116B93
:101D0000103504E20F510008000E105507E30E35A0
:101D100004E20D510008000E0E5528E200C1E6FF56
:101D200001C1E6FF1EEC00F0E552E552F3CF0BF7E0
:101D3000F4CF0CF7090EE66E8EEC00F0E5520FC7FB
:101D4000E6FF10C7E6FF60EC02F0E552E552090E2F
:101D5000E66E8EEC00F0E5520DC7E6FF0EC7E6FF1B
:101D600060EC02F0E552E5529EEC00F00701146BC6
:101D7000156B7A51EA6A000FE96E060EEA22EF50FF
:101D8000836E740EE96E070EEA6E7851EE24786F5A
:101D90007951EE20796F7A51EE207A6F7B51EE20E7
:101DA0007B6F1151E6E0C40EE66E090EE66EE66A40
:101DB000E66A52EC07F0E552E552E552E55264D48A
:101DC0001200279E08D0279E1FAE05D01E6C1F1E36
:101DD000E86A1F22278E1FC019F01EC018F02B6A58
:101DE0002A6A8E0E1A6E1B6A51EF11F0279E0CD0D4
:101DF000279E1FAE09D01C6C1D1E1E1E1F1EE86AEA
:101E00001D221E221F22278E1FC019F01EC018F08F
:101E10001DC02BF01CC02AF09E0E1A6E1B6A51EFDB
:101E200011F0257E276A8DEC11F0A5EC11F027B694
:101E300035EF11F027A20AD027AA03D027BE35EF2D
:101E400011F027A441EF11F03EEF11F027AA05D0C1
:101E500027AC41EF11F03EEF11F027A00AD027A8E0
:101E600008D027BE04D027A402D04AEF11F04EEFCD
:101E700011F02A6A1B6A2550205C296E10E31DC0F0
:101E80002BF01EC018F01FC019F020C028F022C08F
:101E90001DF023C01EF024C01FF0273A09D022C035
:101EA0002BF023C018F024C019F025C028F0296CAD
:101EB000279E27BC278E28C01AF027B07DEF11F08F
:101EC0001A0E29607DEF11F01A6A206A27A408D043
:101ED0001D6C1E1E1F1E201EE86A1E221F222022AD
:101EE00027AC08D02B6C181E191E1A1EE86A18227F
:101EF00019221A221C6A295207E020341F321E328E
:101F00001D321C32292EF9D71D502B261E501822A7
:101F10001F50192220501A221CC02AF0279E1AAEE8
:101F20000BD02A6C2B1E181E191E1A1EE86A2B22B3
:101F3000182219221A22278E1AA006D0D880193208
:101F400018322B322A32282A28C01AF051EF11F009
:101F5000276A8DEC11F0A5EC11F027B635EF11F0E2
:101F600027A205D027BA35EF11F03CEF11F027BAC0
:101F700048EF11F027A005D027B835EF11F048EF52
:101F800011F027B83CEF11F01B6A7F0E20241A6E67
:101F9000E86A1B2225501A5EE86A1B5A1A0E286E40
:101FA000206A2A6A2B6A186A196A22501D5E235019
:101FB0001E5A24501F5A000E205A09E722501D268F
:101FC00023501E2224501F22000E202201D02A8AD4
:101FD000D8901D361E361F362036D8902A362B361E
:101FE00018361936282EE1D71F501E101D10D8A400
:101FF0002A8A51EF11F0276A8DEC11F0A5EC11F04F
:1020000027B635EF11F027A205D027B835EF11F02C
:102010003CEF11F027AA05D027B035EF11F03CEFC7
:1020200011F027B002D027A802D048EF11F01B6AA8
:10203000255020241A6EE86A1B227E0E1A5EE86A7A
:102040001B5A2A6A2B6A186A196A24501F02F4CF95
:1020500019F0F3CF18F023501F02F3502B26F45041
:102060001822000E192224501E02F3502B26F45081
:102070001822000E192222501F02F3502A26F45073
:102080002B22000E1822192223501E02F3502A265A
:10209000F4502B22000E1822192224501D02F35056
:1020A0002A26F4502B22000E1822192222501E023A
:1020B000F4502A26000E2B221822192223501D022A
:1020C000F4502A26000E2B221822192251EF11F06B
:1020D000276A8DEC11F027B672EF10F027A20ED010
:1020E00027B405D07F0E1F6EFF0E1E6E1FD0800E10
:1020F0001F6E1E6A1BD01F6A1E6A18D027B0FBD73E
:102100008F0E2060EDD77E0E2064F5D78E0E205CFA
:1021100005E0D8901F321E32202AF8D727A406D017
:102120001E6C1F1EE86A1F221FAEE5D71200276A29
:102130008DEC11F027B6A1EF10F027A20FD027B435
:1021400007D07F0E1F6EFF0E1E6E1D6E1C6E25D0FB
:10215000800E1F6E01D01F6A000EF6D727B0FBD786
:102160001C6A9F0E2060EBD77E0E2064F4D79E0E73
:10217000205C07E0D8901F321E321D321C32202A0C
:10218000F6D727A40AD01C6C1D1E1E1E1F1EE86A4F
:102190001D221E221F221FAEDED71200E0EC10F01F
:1021A00027B6000C27B0000C27B4000C010CE0ECA3
:1021B00010F027B6000C27B0000C27A4000C010C6F
:1021C000276A8DEC11F0A5EC11F027B6120027AEAE
:1021D00008D027A004D027A802D02780120027907B
:1021E00012002550205C0BE124501F5C08E12350B5
:1021F0001E5C05E122501D5C02E127801200D8A080
:1022000002D0278E10D0205025C020F0256E1F5000
:1022100024C01FF0246E1E5023C01EF0236E1D50DC
:1022200022C01DF0226E2550205C10E0FF0F09E057
:10223000279027B403D027AE2784120027AE279417
:102240001200252AD89024322332223222501D5ED9
:1022500023501E5A24501F5A1FBEEAD7D8901D364D
:102260001E361F36202EF8D7C8D77F0E206EFF0EE1
:102270001F6E1E6E1D6E12007F0E27BEFF0E206E9B
:1022800002D07F0E206E800E1F6E1E6A1D6AF3D76D
:1022900027AE04D0800E206E1F6AF7D7206A1F6A0F
:1022A000F4D7195018102B102A10F8E01BBEF0D7E5
:1022B00019BE0CD01A501B10EBE0D8902A362B36E2
:1022C000183619361A06D8A01B06F2D71B50D4E1CF
:1022D0001A28D2E02AAE11D07F0E2A1402E12BA0D8
:1022E0000CD02B2AE86A1822192207E3D880193269
:1022F00018322B321A2A1A28BFE01A50C9E02BC014
:102300001DF018C01EF019341F6E1A30206E1F32D7
:10231000209E27BE208E3BEF11F01F36203602E3B1
:102320002784277E06E12780206A1F6A1E6A1D6AAD
:102330001200202803E0D8801F321200D8901F32EC
:1023400002E127821200278612002436253602E396
:10235000278C277E06E12788256A246A236A226A59
:102360001200252803E0D88024321200D8902432AD
:10237000EAE1278A1200808285888B8E9194979A51
:102380009DA0A2A5A8ABADB0B3B5B8BBBDC0C2C53A
:10239000C7C9CCCED0D2D4D6D8DADCDEE0E2E3E5D1
:1023A000E6E8E9EBECEDEEEFF0F1F2F3F4F5F5F63B
:1023B000F6F7F7F7F7F7F8F7F7F7F7F7F6F6F5F5B3
:1023C000F4F3F2F1F0EFEEEDECEBE9E8E6E5E3E251
:1023D000E0DEDCDAD8D6D4D2D0CECCC9C7C5C2C0F4
:1023E000BDBBB8B5B3B0ADABA8A5A2A09D9A97945C
:1023F000918E8B888582807D7A7774716E6B68652B
:10240000625F5D5A5754524F4C4A4744423F3D3AEF
:10241000383633312F2D2B29272523211F1D1C1A38
:1024200019171614131211100F0E0D0C0B0A0A09AE
:1024300009080808080808080808080809090A0A15
:102440000B0C0D0E0F10111213141617191A1C1D58
:102450001F21232527292B2D2F313336383A3D3F95
:102460004244474A4C4F5254575A5D5F6265686B0D
:102470006E7174777A7D0808090A0B0C0D0E0F1027
:10248000111213141516171718191A1B1C1D1E1FCD
:1024900020212223242526262728292A2B2C2D2ECD
:1024A0002F30313233343535363738393A3B3C3DCD
:1024B0003E3F40414243444445464748494A4B4CCD
:1024C0004D4E4F50515253535455565758595A5BCD
:1024D0005C5D5E5F60616262636465666768696ACD
:1024E0006B6C6D6E6F7071717273747576777879CD
:1024F0007A7B7C7D7E7F80808182838485868788CD
:10250000898A8B8C8D8E8F8F9091929394959697CC
:1025100098999A9B9C9D9E9E9FA0A1A2A3A4A5A6CC
:10252000A7A8A9AAABACADADAEAFB0B1B2B3B4B5CC
:10253000B6B7B8B9BABBBCBCBDBEBFC0C1C2C3C4CC
:10254000C5C6C7C8C9CACBCBCCCDCECFD0D1D2D3CC
:10255000D4D5D6D7D8D9DADADBDCDDDEDFE0E1E2CC
:10256000E3E4E5E6E7E8E9E9EAEBECEDEEEFF0F1CC
:10257000F2F3F4F5F6F7FFFFFFFFFFFFFFFFFFFFAA
:10258000FFFFFFFFFFFFFFFFFFFFFFFFFFFFFFFF5B
:10259000FFFFFFFFFFFFFFFFFFFFFFFFFFFFFFFF4B
:1025A000FFFFFFFFFFFFFFFFFFFFFFFFFFFFFFFF3B
:1025B000FFFFFFFFFFFFFFFFFFFFFFFFFFFFFFFF2B
:1025C000FFFFFFFFFFFFFFFFFFFFFFFFFFFFFFFF1B
:1025D000FFFFFFFFFFFFFFFFFFFFFFFFFFFFFFFF0B
:1025E000FFFFFFFFFFFFFFFFFFFFFFFFFFFFFFFFFB
:1025F000FFFFFFFFFFFF00000000000000000000E1
:1026000000000000000000000000000000000000CA
:1026100000000000000000000000000000000000BA
:1026200000000000000000000000000000000000AA
:10263000000000000000000000000000000000009A
:10264000000000000000000000000000000000008A
:10265000000000000000000000000000000000007A
:10266000000000000000000000000000000000006A
:1026700000000000000008090B0D0F1113151718BA
:102680001A1C1E2022242627292B2D2F31333536C4
:10269000383A3C3E4042444547494B4D4F515354D4
:1026A00056585A5C5E6062636567696B6D6F7172E4
:1026B0007476787A7C7E8081838587898B8D8F90F4
:1026C000929496989A9C9E9FA1A3A5A7A9ABADAE04
:1026D000B0B2B4B6B8BABCBDBFC1C3C5C7C9CBCC14
:1026E000CED0D2D4D6D8DADBDDDFE1E3E5E7E9EA24
:1026F000ECEEF0F2F4F6F8F6F4F2F0EEECEAE9E7DC
:10270000E5E3E1DFDDDBDAD8D6D4D2D0CECCCBC95D
:10271000C7C5C3C1BFBDBCBAB8B6B4B2B0AEADAB2D
:10272000A9A7A5A3A19F9E9C9A98969492908F8DFD
:102730008B8987858381807E7C7A78767472716FCD
:102740006D6B6967656362605E5C5A58565453519D
:102750004F4D4B4947454442403E3C3A383635336D
:10276000312F2D2B2927262422201E1C1A1817153D
:1027700013110F0D0B094CD8B43C4672616D6520E6
:10278000457272657572206574204F766572666C4D
:102790006F7720646574656374696F6E203A2000FA
:1027A000506F727420636F6D6D2033383430306237
:1027B0006473206F7576657274004D617271756512
:1027C00072203225206475207369676E616C004544
:1027D000534320706F757220736F727469720D00AD
:1027E00043617074757265205461757820737572D9
:1027F00020414443302000536F72746965204E6F4E
:10280000726D616C6520646520507267006361724F
:102810002072656375203A00557361676520513DEC
:1028200031304D687A2078342028504C4C290D00E6
:10283000457272657572205361697369652E2E2E1B
:102840002E2E0D00496E697420436F6E73467265BB
:102850007120314B687A0900466163746575722096
:10286000444453203D2000436F6E7369676E6520BA
:1028700076696120436C61766965720D00566572F8
:1028800073696F6E20312E2E3430303030487A200C
:102890000D004331383A31384634364B32325F44DA
:1028A00044535F5354435844524D5F3132303433B4
:1028B000305F31687A5F34304B687A5F4331382E4D
:1028C000630D00FFFF0EE3CFEAFFE552FF0EE3CFFB
:1028D000E9FFE552E66AE66AE66AE66AD9CFE6FF0C
:1028E000DACFE6FFFA0EE124D96EFF0EE220DA6EAF
:1028F000E66AE66AE66AE66AE66A200EEF5C06E0E9
:10290000090EEF5C03E0EF6603D06BD0EE50F5D715
:102910002D0EEF5C03E1FF0EE32A03D02B0EEF5CDC
:1029200001E1EE502F0EEF6444D03A0EEF6041D03B
:10293000D890F50EE336F60EE336F70EE336F80ED2
:10294000E336FB0EDECFE3FFFC0EDECFE3FFFD0E32
:10295000DECFE3FFFE0EDDCFE3FFDD52DD52D89088
:10296000F50EE336F60EE336F70EE336F80EE336F1
:10297000D890F50EE336F60EE336F70EE336F80E92
:10298000E336FB0EE350DE26FC0EE350DE22FD0EA6
:10299000E350DE22FE0EE350DD22DD52DD52300E2A
:1029A000EE5CDE26000EDE22DE22DD22DD52DD526E
:1029B000B9D7FF0EE3CFE8FFE85213E0F50EE31EB0
:1029C000F60EE31EF70EE31EF80EE31EF50EE32AE5
:1029D00008E1F60EE32A05E1F70EE32A02E1F80E1C
:1029E000E32AE552E552E552E552E552D9CFE9FF37
:1029F000DACFEAFFEECF1CF0EECF1DF0EECF1EF0E7
:102A0000EFCF1FF0FF0EE3CFDAFFE552FF0EE3CF6B
:102A1000D9FFE552E552E5521200D9CFE6FFDACFF1
:102A2000E6FFFA0EE3CFD9FFFB0EE3CFDAFFFD0E90
:102A3000E35209E72D0EDE6EFC0EE31EE32AFD0EC7
:102A4000D8B4E306E31EE652E652E652FD0EE12458
:102A5000E76EFF0EE220E46EE652F70EE3CFE6FFEC
:102A6000F70EE3CFE6FF7DEC15F0F90EE124E96EF9
:102A7000FF0EE220EA6E6DEC15F00AE16AEC15F04B
:102A800009E16DEC15F008E16AEC15F007E108D0FA
:102A900078EC15F073EC15F078EC15F073EC15F09C
:102AA00078EC15F0DE6AF90EE126FF0EE222FF0E49
:102AB000E3CFDAFFE552FF0EE3CFD9FFE552FC0E7C
:102AC000E124E96EFF0EE220EA6EEECFF3FFEFCFD6
:102AD000F4FF1200EF380F0B1200EF500F0B02E162
:102AE000EE52D8841200EF380F0B300FDE6E12005A
:102AF000EE500F0B300FDE6E1200FC0EE3CFE9FF3D
:102B0000FD0EE3CFEAFF100EE66EEE6AEE6AEF6AA4
:102B1000D890FD0EE336FE0EE336ED36ED36EF3699
:102B2000FF0EE30609E09EEC15F0EE529EEC15F068
:102B3000EE529EEC15F0EDD7E56E1200030EEF2479
:102B4000E8B6EF6E300EEF24E8BEEF6E000CD9CF82
:102B5000E6FFDACFE6FFF80EE3CFD9FFF90EE3CFB9
:102B6000DAFFE652E652E652E652E652FB0EE12466
:102B7000E76EFF0EE220E46EE652F30EE3CFE6FFCF
:102B8000F30EE3CFE6FFF30EE3CFE6FFF30EE3CF62
:102B9000E6FF2CEC16F0F50EE124E96EFF0EE220C4
:102BA000EA6E19EC16F019E11CEC16F018E119ECBC
:102BB00016F017E11CEC16F016E119EC16F015E111
:102BC0001CEC16F014E119EC16F013E11CEC16F0F5
:102BD00012E119EC16F011E112D022EC16F027ECFC
:102BE00016F022EC16F027EC16F022EC16F027EC8B
:102BF00016F022EC16F027EC16F022EC16F027EC7B
:102C000016F0DE6AF50EE126FF0EE222FF0EE3CF9C
:102C1000DAFFE552FF0EE3CFD9FFE552FA0EE124C9
:102C2000E96EFF0EE220EA6EEECFF3FFEFCFF4FF86
:102C30001200EF380F0B1200EF500F0B02E1EE52B3
:102C4000D8841200EF380F0B300FDE6E1200EE50FA
:102C50000F0B300FDE6E1200FA0EE3CFE9FFFB0E12
:102C6000E3CFEAFF200EE66EEE6AEE6AEE6AEE6AE7
:102C7000EF6AD890FB0EE336FC0EE336FD0EE3362A
:102C8000FE0EE336ED36ED36ED36ED36EF36FF0E61
:102C9000E3060FE05BEC16F0EE525BEC16F0EE5242
:102CA0005BEC16F0EE525BEC16F0EE525BEC16F0BD
:102CB000E1D7E56E1200030EEF24E8B6EF6E300E9A
:102CC000EF24E8BEEF6E000CD9CFE6FFDACFE6FFC7
:102CD000E1CFD9FFE2CFDAFF130EE12402E3E1688E
:102CE000E652E16E0C0EDB6AD950FA0FE96EFF0E68
:102CF000DA20EA6E080EEECFDBFF090EEECFDBFF27
:102D00000A0EEECFDBFF0B0EEECFDBFF1FD9D95043
:102D1000080F17D9EECFE6FFEECFE6FFEECFE6FFC6
:102D2000EFCFE6FFADEC17F0006E060EE15C02E2BD
:102D3000E16AE552E16E0050DF6E020EDF5C01E0F9
:102D4000BCD0050EDBCF02F0060EDBCF03F0F80E91
:102D5000DB50025C006EF90EDB500358016E7F0EF3
:102D6000005E000E015A0D0E00C0DBFF0E0E01C00A
:102D7000DBFF0D0E0E0EDBCF01F00001800E011403
:102D80000AE0010EF36E0C0EF3CFDBFF070EDB50F3
:102D900001E098D09DD00D0EDBCF00F00E0EDBCF02
:102DA00001F0D890015004E6170E005C000E0158A7
:102DB00001E39ED0046805687F0E066E076A0D0E5B
:102DC000DB501F0B04C000F005C001F006C002F08C
:102DD00007C003F007E0D89003320232013200321C
:102DE000E806F9E10F0E00C0DBFF100E01C0DBFFAB
:102DF000110E02C0DBFF120E03C0DBFF0F0EDBCF94
:102E000000F0100EDBCF01F0110EDBCF02F0120E3E
:102E1000DBCF03F0D950010F94D8EE500016EE50DE
:102E20000116EE500216EE5003160050011002106B
:102E3000031002E1000E01D0010EE76E0C0EE7CF89
:102E4000DBFFDB5055E0046A056A800E066E076AF8
:102E5000010E086E096A0A6A0B6AD9500F0F71D801
:102E6000EE500826EE500922EE500A22EE500B22B8
:102E70000850045C006E09500558016E0A5006584F
:102E8000026E0B500758036ED950010F5AD80050EC
:102E9000EE160150EE160250EE160350EE16D95003
:102EA000080FE66E000EDA20E66E50D83BEC18F004
:102EB000E552E552E552E5521BD0DF0419E1070E59
:102EC000DB5006E0006A016A026A800E036E04D0DD
:102ED000006A016A026A036A080E00C0DBFF090E7D
:102EE00001C0DBFF0A0E02C0DBFF0B0E03C0DBFFDD
:102EF000F60EDBCFE9FFF70EDBCFEAFF0C0EDBCFE0
:102F0000EFFF080EDBCF00F0090EDBCF01F00A0E59
:102F1000DBCF02F00B0EDBCF03F000C01CF001C0D2
:102F20001DF002C01EF003C01FF0130EE15C02E2B0
:102F3000E16AE552E16EE552E5CFDAFFE7CFD9FF6E
:102F40001200E96E000EDA20EA6E1200D950010F6D
:102F5000E66E000EDA20E66E1200D9CFE6FFDACF79
:102F6000E6FFE1CFD9FFE2CFDAFFE6520068016861
:102F70007F0E026E036AD950FA0FE96EFF0EDA2057
:102F8000EA6EEE500016EE500116EE500216EE50AC
:102F900003166AD800C0EEFF01C0EEFF02C0EEFFCC
:102FA00003C0EEFFFD0EDB50800B02E0010E01D0EE
:102FB000000EE66E59D8060EE926000EEA22E5520A
:102FC000E750EF6EFC0EDBCF00F0FD0EDBCF01F023
:102FD000D89000360136FC0E00C0DBFFFD0E01C0AC
:102FE000DBFFDB50E66E40D8040EE926000EEA2235
:102FF000E552E750EE6EED6AFD0EDB50006E016AA1
:10300000FF0E001818E1015016E12ED8EECF00F0A7
:10301000EECF01F0EECF02F0EFCF03F00050011041
:103020000210031006E0210E0F010A6F0B6B800ED9
:103030000BD0040E09D0FD0EDB5008E115D8EE6A66
:10304000EE6AEE6AEE6A010EDF6E06D0020EDF6EE9
:103050000BD8EE52EE52EE8EDF50E552E552E5CF40
:10306000DAFFE7CFD9FF1200F80EDBCFE9FFF90E48
:10307000DBCFEAFF1200D9CFE6FFDACFE6FFE1CFE0
:10308000D9FFE2CFDAFF5BD8013411E20050FE082D
:10309000000E01540CE276D805E06CD8800EEE6E7E
:1030A000EE6847D067D8800EEE6E7F0E0ED047D800
:1030B000D890015004E6010E005C000E01580BE2AE
:1030C00061D805E057D8EE6A800EEE6E32D052D845
:1030D000EE6AEE6A2ED047D8EECF00F0EECF01F0C8
:1030E000EECF02F0EFCF03F032D800C0EEFF01C008
:1030F000EEFF02C0EEFF03C0EEFF21D80050010B2F
:1031000005E025D8020E3AD8EF8E04D020D8020E62
:1031100035D8EF9E14D8D8900132003218D8030E5B
:103120002DD800C0EFFF1AD804E011D8030E26D81E
:10313000EF8EE552E5CFDAFFE7CFD9FF120013D8C3
:10314000040E1CD8EECF00F0EFCF01F01200FA0E03
:10315000DBCFE9FFFB0EDBCFEAFF120004D8060E3F
:103160000DD8EF501200FC0EDBCFE9FFFD0EDBCFD8
:10317000EAFF1200ECDFEE6AEE6A1200E926000EAA
:10318000EA221200220E0F010A6F0B6BAEEF18F04D
:10319000D9CFE6FFDACFE6FFE1CFD9FFE2CFDAFF02
:1031A000060EE12402E3E168E652E16ED950050F14
:1031B000E66E000EDA20E66E000EE66EE66AD95084
:1031C000FA0FE96EFF0EDA20EA6EEECFE6FFEECFE1
:1031D000E6FFEECFE6FFEFCFE6FF64EC16F0006E01
:1031E000080EE15C02E2E16AE552E16E0050010E78
:1031F0001CC0DBFF020E1DC0DBFF030E1EC0DBFF89
:10320000040E1FC0DBFF050EDB502AE0040EDB506E
:10321000800B26E1006A016A800E026E3F0E036E8B
:10322000D950010FE96E000EDA20EA6EEECF1DF0E4
:10323000EECF1EF0EECF1FF0EFCF20F000C022F057
:1032400001C023F002C024F003C025F012EC0FF0FF
:1032500020C0EDFF1FC0EDFF1EC0EDFF1DC0EFFF42
:10326000010EDBCF00F0020EDBCF01F0030EDBCF4F
:1032700002F0040EDBCF03F000C01CF001C01DF013
:1032800002C01EF003C01FF0060EE15C02E2E16A1C
:10329000E552E16EE552E5CFDAFFE7CFD9FF120044
:1032A0000E0EF66E000EF76E000EF86E0F0109009E
:1032B000F550056F0900F550066F03E1056701D071
:1032C0003DD00900F550006F0900F550016F09006D
:1032D000F550026F09000900F550E96E0900F5503C
:1032E000EA6E090009000900F550036F0900F55066
:1032F000046F09000900F6CF07FFF7CF08FFF8CFEA
:1033000009FF00CFF6FF01CFF7FF02CFF8FF0F0153
:10331000035302E1045307E00900F550EE6E030782
:10332000F8E20407F9D707CFF6FF08CFF7FF09CF78
:10333000F8FF0F010507000E065BBFD71200FB0E5A
:10334000E3CFF6FFFC0EE3CFF7FFFD0EE3CFF8FF70
:10335000FE0EE3CFE9FFFF0EE3CFEAFFE9CFF3FF75
:10336000EACFF4FFF90EE35003E1FA0EE35009E06F
:10337000F90EE30602E2FA0EE3060900F5CFEEFFCE
:10338000F1D71200FB0EE3CFF6FFFC0EE3CFF7FF01
:10339000FD0EE3CFF8FFFE0EE3CFE9FFFF0EE3CF14
:1033A000EAFFE9CFF3FFEACFF4FF0900F5CFEFFF23
:1033B000EE66FBD71200FE0EE3CFE9FFFF0EE3CF70
:1033C000EAFFF36AF46AEE5203E0F34AF42AFBD709
:1033D0001200D9CFE6FFDACFE6FFE1CFD9FFE2CF87
:1033E000DAFFAC6AAB6AFD0EDBB0AC88DBA202D0C0
:1033F000AC8CAB8CDBB4AC8EDBA602D0AB8801D03E
:10340000AB8ADBB8AC84DBBAAB86DBAC02D09D8A7E
:1034100001D09D9ADBAE02D09D8801D09D98FB0E15
:10342000DB50AF6EFC0EDBCF01F001C000F0016A93
:103430000050B06EAC8AAB8EE552E5CFDAFFE7CF35
:10344000D9FF12001C502102F3CF18F0F4CF19F06D
:103450002202F3501926000EF4201A6E1C5023028B
:10346000F3501A26000EF4201B6E1C502402F35059
:103470001B261D502102F3501926F4501A22000E6B
:103480001B221D502202F3501A26F4501B221D50FD
:103490002302F3501B261E502102F3501A26F4502B
:1034A0001B221E502202F3501B261F502102F350F4
:1034B0001B261200D9CFE6FFDACFE6FFE1CFD9FF16
:1034C000E2CFDAFFE652F20E0F010C17ABAC03D0DD
:1034D0000C91ABB00C81ABB40C85ABB20C87AE5089
:1034E000DF6EDF50E552E552E5CFDAFFE7CFD9FFD7
:1034F0001200D9CFE6FFDACFE6FFE1CFD9FFE2CF66
:10350000DAFFE652E652FC0EDBCFDEFFDBCFDDFF5B
:10351000010EDB50CF6EDF50CE6EE552E552E55224
:10352000E5CFDAFFE7CFD9FF1200D9CFE6FFDACF38
:10353000E6FFE1CFD9FFE2CFDAFFACAC04D0AC902C
:103540000F010CB3AC80FD0EDB50AD6EE552E5CF44
:10355000DAFFE7CFD9FF1200F36AF46AFF0EE12425
:10356000E96EFF0EE220EA6EED6607D02F0EEF64E3
:1035700004D03A0EEF6001D0F32A1200380EF36E39
:1035800000EE00F00F0E01D81200EA6002D0EE6AE1
:10359000FCD7F350E9601200EE6AFCD71EEE00F093
:1035A0002EEE00F0F86A279C50EC19F003EC00F0C6
:1035B000E3EC08F0FBD71200FF0EE350E84E1200D8
:1035C000000000D000D000D0E82EFAD71200C4507E
:1035D000036E026AC3500210F36E03C0F4FF1200C0
:1035E000C250020B01E0010E1200C28212007A27C3
:1035F000A027BA27CF27E027F7270D28182830283B
:103600004428582867287D289228762350524F4A0C
:1036100045543A2031384634364B32325F444453B5
:103620002E6D6370200D00000000000000000000FF
:10363000000000000000000000000000000000008A
:103640000000000000000000000000001E013132F8
:10365000333435363738393031323334350031325E
:10366000333435363738393031323334353600007B
:10367000000000000000000000000000000000004A
:10368000000000000000000000000000000000003A
:10369000FFFFFFFFFFFFFFFFFFFFFFFFFFFFFFFF3A
:1036A000FFFFFFFFFFFFFFFFFFFFFFFFFFFFFFFF2A
:0200000400F00A
:100000002031384634364B32322034304D687A2035
:1000100031304D487A7834202020504C4C0D00006F
:100020002053696E7573207375722031207065726C
:10003000696F6465202E2E2E2E2E2020200D0000AC
:100040002043617272652073757220312070657271
:10005000696F64652020202020202020200D0000D2
:1000600020547269616E676C65207375722031204F
:10007000706572696F646520202E2020200D0000BD
:100080002044656E742064652073636965202F20A9
:100090003120706572696F64652020200D000000BA
:1000A00020526576657273652064656E74206465A0
:1000B0002073636965202F2031207065720D000068
:1000C00020416363657320617520546175782076E3
:1000D0006961205820657420506F7461722020205F
:1000E00020566F69653020706F757220312F323560
:1000F00036202061203235352F32353620200D0054
:10010000204D61727175657572202B2D3438706FBA
:10011000696E747320737572203438200D000000EE
:10012000204D504C4142204944452056382E38330A
:100130002C4331382056332E34302E2020200D0011
:10014000FFFFFFFFFFFFFFFFFFFFFFFFFFFFFFFFBF
:10015000FFFFFFFFFFFFFFFFFFFFFFFFFFFFFFFFAF
:10016000FFFFFFFFFFFFFFFFFFFFFFFFFFFFFFFF9F
:10017000FFFFFFFFFFFFFFFFFFFFFFFFFFFFFFFF8F
:020000040030CA
:0E0000000032183C009984000FC00FE00F4042
:020000040020DA
:08000000FFFFFFFFFFFFFFFF00
:00000001FF
